:1006A7000800080308060809080C080F08120815AF
:1006B7000819081C081F082208250828082B082FD6
:1006C700083208350838083B083E084108450848FD
:1006D700084B084E085108540857085B085E086124
:1006E70008640867086A086D087108740877087A4B
:1006F700087D088008830886088A088D0890089373
:1007070008960899089C08A008A308A608A908AC99
:1007170008AF08B208B508B908BC08BF08C208C5C1
:1007270008C808CB08CE08D208D508D808DB08DEE9
:1007370008E108E408E708EB08EE08F108F408F711
:1007470008FA08FD090009040907090A090D091033
:10075700091309160919091C09200923092609295A
:10076700092C092F093209350938093C093F094283
:1007770009450948094B094E095109540957095BAD
:10078700095E096109640967096A096D09700973D6
:1007970009760979097D0980098309860989098C00
:1007A700098F099209950998099B099E09A209A52C
:1007B70009A809AB09AE09B109B409B709BA09BD56
:1007C70009C009C309C609C909CC09D009D309D683
:1007D70009D909DC09DF09E209E509E809EB09EEAE
:1007E70009F109F409F709FA09FD0A000A030A06DB
:1007F7000A090A0D0A100A130A160A190A1C0A1FFF
:100807000A220A250A280A2B0A2E0A310A340A372D
:100817000A3A0A3D0A400A430A460A490A4C0A4F5D
:100827000A520A550A580A5B0A5E0A610A640A678D
:100837000A6A0A6D0A700A730A760A790A7C0A7FBD
:100847000A820A850A880A8B0A8E0A910A940A97ED
:100857000A9A0A9D0AA00AA30AA60AA90AAC0AAE1E
:100867000AB10AB40AB70ABA0ABD0AC00AC30AC655
:100877000AC90ACC0ACF0AD20AD50AD80ADB0ADE85
:100887000AE10AE30AE60AE90AEC0AEF0AF20AF5BC
:100897000AF80AFB0AFE0B010B040B070B090B0CEA
:1008A7000B0F0B120B150B180B1B0B1E0B210B241D
:1008B7000B260B290B2C0B2F0B320B350B380B3B55
:1008C7000B3D0B400B430B460B490B4C0B4F0B518E
:1008D7000B540B570B5A0B5D0B600B630B650B68C7
:1008E7000B6B0B6E0B710B740B760B790B7C0B7F01
:1008F7000B820B850B870B8A0B8D0B900B930B953C
:100907000B980B9B0B9E0BA10BA40BA60BA90BAC77
:100917000BAF0BB10BB40BB70BBA0BBD0BBF0BC2B5
:100927000BC50BC80BCA0BCD0BD00BD30BD60BD8F3
:100937000BDB0BDE0BE10BE30BE60BE90BEB0BEE33
:100947000BF10BF40BF60BF90BFC0BFF0C010C0472
:100957000C070C090C0C0C0F0C120C140C170C1AAE
:100967000C1C0C1F0C220C240C270C2A0C2D0C2FF2
:100977000C320C350C370C3A0C3D0C3F0C420C4535
:100987000C470C4A0C4C0C4F0C520C540C570C5A7D
:100997000C5C0C5F0C620C640C670C690C6C0C6FC4
:1009A7000C710C740C770C790C7C0C7E0C810C840C
:1009B7000C860C890C8B0C8E0C900C930C960C9857
:1009C7000C9B0C9D0CA00CA20CA50CA80CAA0CADA2
:1009D7000CAF0CB20CB40CB70CB90CBC0CBE0CC1F0
:1009E7000CC30CC60CC90CCB0CCE0CD00CD30CD53D
:1009F7000CD80CDA0CDD0CDF0CE20CE40CE70CE98C
:100A07000CEB0CEE0CF00CF30CF50CF80CFA0CFDDF
:100A17000CFF0D020D040D070D090D0B0D0E0D102A
:100A27000D130D150D180D1A0D1C0D1F0D210D247D
:100A37000D260D280D2B0D2D0D300D320D340D37D4
:100A47000D390D3C0D3E0D400D430D450D470D4A2B
:100A57000D4C0D4E0D510D530D560D580D5A0D5D84
:100A67000D5F0D610D640D660D680D6A0D6D0D6FDF
:100A77000D710D740D760D780D7B0D7D0D7F0D813C
:100A87000D840D860D880D8A0D8D0D8F0D910D949A
:100A97000D960D980D9A0D9D0D9F0DA10DA30DA5FA
:100AA7000DA80DAA0DAC0DAE0DB10DB30DB50DB75B
:100AB7000DB90DBC0DBE0DC00DC20DC40DC60DC9BF
:100AC7000DCB0DCD0DCF0DD10DD30DD60DD80DDA24
:100AD7000DDC0DDE0DE00DE20DE50DE70DE90DEB8B
:100AE7000DED0DEF0DF10DF30DF50DF70DFA0DFCF5
:100AF7000DFE0E000E020E040E060E080E0A0E0C58
:100B07000E0E0E100E120E140E160E180E1B0E1DC4
:100B17000E1F0E210E230E250E270E290E2B0E2D2E
:100B27000E2F0E310E330E350E370E390E3B0E3C9F
:100B37000E3E0E400E420E440E460E480E4A0E4C16
:100B47000E4E0E500E520E540E560E580E5A0E5B87
:100B57000E5D0E5F0E610E630E650E670E690E6BFE
:100B67000E6C0E6E0E700E720E740E760E780E7977
:100B77000E7B0E7D0E7F0E810E830E840E860E88F1
:100B87000E8A0E8C0E8E0E8F0E910E930E950E966C
:100B97000E980E9A0E9C0E9E0E9F0EA10EA30EA5EA
:100BA7000EA60EA80EAA0EAC0EAD0EAF0EB10EB26B
:100BB7000EB40EB60EB80EB90EBB0EBD0EBE0EC0ED
:100BC7000EC20EC30EC50EC70EC80ECA0ECC0ECD72
:100BD7000ECF0ED10ED20ED40ED60ED70ED90EDBF7
:100BE7000EDC0EDE0EDF0EE10EE30EE40EE60EE780
:100BF7000EE90EEA0EEC0EEE0EEF0EF10EF20EF40B
:100C07000EF50EF70EF90EFA0EFC0EFD0EFF0F0095
:100C17000F020F030F050F060F080F090F0B0F0C1D
:100C27000F0E0F0F0F110F120F140F150F160F18AE
:100C37000F190F1B0F1C0F1E0F1F0F210F220F2342
:100C47000F250F260F280F290F2A0F2C0F2D0F2FD7
:100C57000F300F310F330F340F350F370F380F3A6F
:100C67000F3B0F3C0F3E0F3F0F400F420F430F4408
:100C77000F450F470F480F490F4B0F4C0F4D0F4FA5
:100C87000F500F510F520F540F550F560F570F5943
:100C97000F5A0F5B0F5C0F5E0F5F0F600F610F62E4
:100CA7000F640F650F660F670F680F6A0F6B0F6C86
:100CB7000F6D0F6E0F6F0F710F720F730F740F752C
:100CC7000F760F770F790F7A0F7B0F7C0F7D0F7ED3
:100CD7000F7F0F800F810F820F840F850F860F877D
:100CE7000F880F890F8A0F8B0F8C0F8D0F8E0F8F29
:100CF7000F900F910F920F930F940F950F960F97D9
:100D07000F980F990F9A0F9B0F9C0F9D0F9E0F9F88
:100D17000FA00FA10FA20FA30FA40FA50FA50FA63A
:100D27000FA70FA80FA90FAA0FAB0FAC0FAD0FAEF0
:100D37000FAE0FAF0FB00FB10FB20FB30FB40FB4A9
:100D47000FB50FB60FB70FB80FB90FB90FBA0FBB63
:100D57000FBC0FBD0FBD0FBE0FBF0FC00FC10FC11F
:100D67000FC20FC30FC40FC40FC50FC60FC70FC7DE
:100D77000FC80FC90FCA0FCA0FCB0FCC0FCC0FCD9F
:100D87000FCE0FCE0FCF0FD00FD00FD10FD20FD264
:100D97000FD30FD40FD40FD50FD60FD60FD70FD829
:100DA7000FD80FD90FD90FDA0FDB0FDB0FDC0FDCF2
:100DB7000FDD0FDD0FDE0FDF0FDF0FE00FE00FE1BD
:100DC7000FE10FE20FE20FE30FE30FE40FE40FE58C
:100DD7000FE50FE60FE60FE70FE70FE80FE80FE95C
:100DE7000FE90FEA0FEA0FEB0FEB0FEC0FEC0FEC2D
:100DF7000FED0FED0FEE0FEE0FEF0FEF0FEF0FF001
:100E07000FF00FF00FF10FF10FF20FF20FF20FF3D8
:100E17000FF30FF30FF40FF40FF40FF50FF50FF5B2
:100E27000FF60FF60FF60FF70FF70FF70FF70FF88D
:100E37000FF80FF80FF80FF90FF90FF90FF90FFA6D
:100E47000FFA0FFA0FFA0FFB0FFB0FFB0FFB0FFB4E
:100E57000FFC0FFC0FFC0FFC0FFC0FFD0FFD0FFD30
:100E67000FFD0FFD0FFD0FFD0FFE0FFE0FFE0FFE17
:100E77000FFE0FFE0FFE0FFE0FFF0FFF0FFF0FFFFF
:100E87000FFF0FFF0FFF0FFF0FFF0FFF0FFF0FFFEB
:100E97000FFF0FFF0FFF0FFF0FFF0FFF0FFF0FFFDB
:100EA7000FFF0FFF0FFF0FFF0FFF0FFF0FFF0FFFCB
:100EB7000FFF0FFF0FFF0FFF0FFF0FFF0FFF0FFFBB
:100EC7000FFF0FFF0FFF0FFF0FFF0FFE0FFE0FFEAE
:100ED7000FFE0FFE0FFE0FFE0FFE0FFD0FFD0FFDA6
:100EE7000FFD0FFD0FFD0FFD0FFC0FFC0FFC0FFC9F
:100EF7000FFC0FFB0FFB0FFB0FFB0FFB0FFA0FFA9C
:100F07000FFA0FFA0FF90FF90FF90FF90FF80FF89A
:100F17000FF80FF80FF70FF70FF70FF70FF60FF69A
:100F27000FF60FF50FF50FF50FF40FF40FF40FF39E
:100F37000FF30FF30FF20FF20FF20FF10FF10FF0A4
:100F47000FF00FF00FEF0FEF0FEF0FEE0FEE0FEDAC
:100F57000FED0FEC0FEC0FEC0FEB0FEB0FEA0FEAB7
:100F67000FE90FE90FE80FE80FE70FE70FE60FE6C6
:100F77000FE50FE50FE40FE40FE30FE30FE20FE2D6
:100F87000FE10FE10FE00FE00FDF0FDF0FDE0FDDE7
:100F97000FDD0FDC0FDC0FDB0FDB0FDA0FD90FD9FB
:100FA7000FD80FD80FD70FD60FD60FD50FD40FD412
:100FB7000FD30FD20FD20FD10FD00FD00FCF0FCE2D
:100FC7000FCE0FCD0FCC0FCC0FCB0FCA0FCA0FC947
:100FD7000FC80FC70FC70FC60FC50FC40FC40FC366
:100FE7000FC20FC10FC10FC00FBF0FBE0FBD0FBD87
:100FF7000FBC0FBB0FBA0FB90FB90FB80FB70FB6AA
:101007000FB50FB40FB40FB30FB20FB10FB00FAFCF
:101017000FAE0FAE0FAD0FAC0FAB0FAA0FA90FA8F6
:101027000FA70FA60FA50FA50FA40FA30FA20FA120
:101037000FA00F9F0F9E0F9D0F9C0F9B0F9A0F994D
:101047000F980F970F960F950F940F930F920F917D
:101057000F900F8F0F8E0F8D0F8C0F8B0F8A0F89AD
:101067000F880F870F860F850F840F820F810F80E0
:101077000F7F0F7E0F7D0F7C0F7B0F7A0F790F7716
:101087000F760F750F740F730F720F710F6F0F6E4F
:101097000F6D0F6C0F6B0F6A0F680F670F660F6589
:1010A7000F640F620F610F600F5F0F5E0F5C0F5BC6
:1010B7000F5A0F590F570F560F550F540F520F5105
:1010C7000F500F4F0F4D0F4C0F4B0F490F480F4746
:1010D7000F450F440F430F420F400F3F0F3E0F3C8A
:1010E7000F3B0F3A0F380F370F350F340F330F31D0
:1010F7000F300F2F0F2D0F2C0F2A0F290F280F2618
:101107000F250F230F220F210F1F0F1E0F1C0F1B61
:101117000F190F180F160F150F140F120F110F0FAE
:101127000F0E0F0C0F0B0F090F080F060F050F03FC
:101137000F020F000EFF0EFD0EFC0EFA0EF90EF752
:101147000EF50EF40EF20EF10EEF0EEE0EEC0EEAA9
:101157000EE90EE70EE60EE40EE30EE10EDF0EDEFD
:101167000EDC0EDB0ED90ED70ED60ED40ED20ED154
:101177000ECF0ECD0ECC0ECA0EC80EC70EC50EC3AF
:101187000EC20EC00EBE0EBD0EBB0EB90EB80EB609
:101197000EB40EB20EB10EAF0EAD0EAC0EAA0EA867
:1011A7000EA60EA50EA30EA10E9F0E9E0E9C0E9AC6
:1011B7000E980E960E950E930E910E8F0E8E0E8C28
:1011C7000E8A0E880E860E840E830E810E7F0E7D8C
:1011D7000E7B0E790E780E760E740E720E700E6EF2
:1011E7000E6C0E6B0E690E670E650E630E610E5F59
:1011F7000E5D0E5B0E5A0E580E560E540E520E50C2
:101207000E4E0E4C0E4A0E480E460E440E420E402F
:101217000E3E0E3C0E3B0E390E370E350E330E3199
:101227000E2F0E2D0E2B0E290E270E250E230E2107
:101237000E1F0E1D0E1B0E180E160E140E120E107C
:101247000E0E0E0C0E0A0E080E060E040E020E00EF
:101257000DFE0DFC0DFA0DF70DF50DF30DF10DEF6C
:101267000DED0DEB0DE90DE70DE50DE20DE00DDEE2
:101277000DDC0DDA0DD80DD60DD30DD10DCF0DCD5B
:101287000DCB0DC90DC60DC40DC20DC00DBE0DBCD5
:101297000DB90DB70DB50DB30DB10DAE0DAC0DAA52
:1012A7000DA80DA50DA30DA10D9F0D9D0D9A0D98D0
:1012B7000D960D940D910D8F0D8D0D8A0D880D8650
:1012C7000D840D810D7F0D7D0D7B0D780D760D74D1
:1012D7000D710D6F0D6D0D6A0D680D660D640D6155
:1012E7000D5F0D5D0D5A0D580D560D530D510D4ED9
:1012F7000D4C0D4A0D470D450D430D400D3E0D3C60
:101307000D390D370D340D320D300D2D0D2B0D28E8
:101317000D260D240D210D1F0D1C0D1A0D180D1571
:101327000D130D100D0E0D0B0D090D070D040D02FC
:101337000CFF0CFD0CFA0CF80CF50CF30CF00CEE92
:101347000CEB0CE90CE70CE40CE20CDF0CDD0CDA1F
:101357000CD80CD50CD30CD00CCE0CCB0CC90CC6AE
:101367000CC30CC10CBE0CBC0CB90CB70CB40CB242
:101377000CAF0CAD0CAA0CA80CA50CA20CA00C9DD4
:101387000C9B0C980C960C930C900C8E0C8B0C8968
:101397000C860C840C810C7E0C7C0C790C770C74FD
:1013A7000C710C6F0C6C0C690C670C640C620C5F95
:1013B7000C5C0C5A0C570C540C520C4F0C4C0C4A2E
:1013C7000C470C450C420C3F0C3D0C3A0C370C35C6
:1013D7000C320C2F0C2D0C2A0C270C240C220C1F62
:1013E7000C1C0C1A0C170C140C120C0F0C0C0C09FF
:1013F7000C070C040C010BFF0BFC0BF90BF60BF4A1
:101407000BF10BEE0BEB0BE90BE60BE30BE10BDE42
:101417000BDB0BD80BD60BD30BD00BCD0BCA0BC8E2
:101427000BC50BC20BBF0BBD0BBA0BB70BB40BB184
:101437000BAF0BAC0BA90BA60BA40BA10B9E0B9B25
:101447000B980B950B930B900B8D0B8A0B870B85CA
:101457000B820B7F0B7C0B790B760B740B710B6E6E
:101467000B6B0B680B650B630B600B5D0B5A0B5714
:101477000B540B510B4F0B4C0B490B460B430B40BB
:101487000B3D0B3B0B380B350B320B2F0B2C0B2962
:101497000B260B240B210B1E0B1B0B180B150B120A
:1014A7000B0F0B0C0B090B070B040B010AFE0AFBB6
:1014B7000AF80AF50AF20AEF0AEC0AE90AE60AE369
:1014C7000AE10ADE0ADB0AD80AD50AD20ACF0ACC11
:1014D7000AC90AC60AC30AC00ABD0ABA0AB70AB4C1
:1014E7000AB10AAE0AAC0AA90AA60AA30AA00A9D6B
:1014F7000A9A0A970A940A910A8E0A8B0A880A8519
:101507000A820A7F0A7C0A790A760A730A700A6DC8
:101517000A6A0A670A640A610A5E0A5B0A580A5578
:101527000A520A4F0A4C0A490A460A430A400A3D28
:101537000A3A0A370A340A310A2E0A2B0A280A25D8
:101547000A220A1F0A1C0A190A160A130A100A0D88
:101557000A090A060A030A0009FD09FA09F709F444
:1015670009F109EE09EB09E809E509E209DF09DCF8
:1015770009D909D609D309D009CC09C909C609C3AC
:1015870009C009BD09BA09B709B409B109AE09AB60
:1015970009A809A509A2099E099B09980995099215
:1015A700098F098C0989098609830980097D0979C9
:1015B700097609730970096D096A09670964096180
:1015C700095E095B095709540951094E094B094836
:1015D70009450942093F093C093809350932092FEC
:1015E700092C0929092609230920091C09190916A3
:1015F70009130910090D090A09070904090008FD5B
:1016070008FA08F708F408F108EE08EB08E708E419
:1016170008E108DE08DB08D808D508D208CE08CBD1
:1016270008C808C508C208BF08BC08B908B508B289
:1016370008AF08AC08A908A608A308A0089C089941
:10164700089608930890088D088A088608830880FA
:10165700087D087A087708740871086D086A0867B2
:1016670008640861085E085B085708540851084E6B
:10167700084B084808450841083E083B0838083524
:101687000832082F082B082808250822081F081CDD
:10169700081908150812080F080C08090806080396
:1016A7001000100B10161021102C10371043104E7D
:1016B700105910651070107B10871092109E10A99A
:1016C70010B510C010CC10D810E310EF10FB1107A5
:1016D7001113111E112A11361142114E115A11669A
:1016E7001172117E118A119711A311AF11BB11C885
:1016F70011D411E011ED11F912061212121F122B5B
:10170700123812451251125E126B1278128412911E
:10171700129E12AB12B812C512D212DF12EC12F9D6
:10172700130613141321132E133C13491356136472
:101737001371137F138C139A13A713B513C313D005
:1017470013DE13EC13FA1408141614231431143F80
:10175700144E145C146A14781486149414A314B1E8
:1017670014BF14CE14DC14EB14F91508151615253F
:101777001534154215511560156F157E158D159C7D
:1017870015AB15BA15C915D815E715F616051615AB
:1017970016241633164316521662167116811690C2
:1017A70016A016B016C016CF16DF16EF16FF170FC6
:1017B700171F172F173F174F175F177017801790AF
:1017C70017A117B117C117D217E217F31804181486
:1017D700182518361847185718681879188A189B43
:1017E70018AC18BE18CF18E018F1190219141925EA
:1017F70019371948195A196B197D198F19A019B278
:1018070019C419D619E819FA1A0C1A1E1A301A42ED
:101817001A551A671A791A8B1A9E1AB01AC31AD54B
:101827001AE81AFB1B0E1B201B331B461B591B6C8C
:101837001B7F1B921BA51BB81BCC1BDF1BF21C06B7
:101847001C191C2D1C401C541C671C7B1C8F1CA3C3
:101857001CB71CCB1CDF1CF31D071D1B1D2F1D43B5
:101867001D581D6C1D801D951DA91DBE1DD31DE78F
:101877001DFC1E111E261E3B1E501E651E7A1E8F46
:101887001EA41EB91ECF1EE41EFA1F0F1F251F3AE6
:101897001F501F661F7B1F911FA71FBD1FD31FE967
:1018A7000A000900080007000600050004000300FD
:0618B70002000100000028
:102EB2004102F54EC10B4102F400410306004102FA
:102EC2003600410301014202EF00014103000141CA
:102ED20002F1064202020000410204004203020023
:102EE20000420304000042023700144203070000BC
:042EF20041023A015E
:1031C800E4F5AB75AB80FF0FEFB4C8FB43ABC0E4CD
:0E31D800FF0FEFB4C8FBE5AB30E5FB75B28727
:0131E60022C6
:1031E700758921758E0C758CFE758A1A75885075D0
:0E31F700C804E4F5CA75CBFEF5CC75CDFE22FA
:1032C50075BC909002F1E0F5BB75E88075BAF72200
:0733100075B9F675B5F42252
:04333100E4F5D122CC
:1032220075E10575E2C075A48075F2C075F3FFE41F
:0C323200F5D675A63875D40375D5FF22BB
:0A32FE0075B80275E60975A8A22252
:10323E00E4F5881231C81232221231E71232C51269
:0B324E0033101233311232FE0230B890
:08310100AB07AF031BEF601ADE
:103109009003AC121FEA0000445C9003AC74FF12F8
:0A3119001FABEC4D4E4F60E280F05A
:013123002289
:102D7A0053D9BF12323E123259123124E4FF7EB4C3
:102D8A0090023B7455F0A3DEFC7E007FB412300D36
:102D9A00EF60FAC2AF90039FE0B414099002F47492
:102DAA0001F01232D590039FE0FFB41505E49002BA
:102DBA00F4F09002F4E06022EF14601304701B90A8
:102DCA0003A0E09003B0F01231241232E4800B9099
:0E2DDA0003A0E09003B0F0121A1BD2AF80AF3E
:0E32E400E51424FFB392A4E51424FF92A32264
:102BCD00A2A2920B9002F5300B05744EF0800374A7
:102BDD004FF0900306E0900236F0E58054409003EC
:102BED0006F0E07036900203E004F07006900202E9
:102BFD00E004F0D3900203E09400900202E094020E
:102C0D0040479002F5E0FF7D081231889002047470
:102C1D0001F0E4900202F0A3F0802EE4900202F0A5
:102C2D00A3F0900236E0701C900204E07016900341
:102C3D0001E070047F0180027F00900301EFF0F549
:102C4D00141232D5E4900204F0E5A054409002F441
:012C5D00F086
:012C5E002253
:031A0600022A3C75
:102A3C00C0E0C083C082C0D075D000C000C006C04A
:012A4C000782
:102A4D00900302E0FEA3E0F596EEF5979002F2E01A
:102A5D00FEA3E0FFC374FF9F900305F0740F9E90DB
:102A6D000304F0E0FEA3E0F5F4EEF5F5900307E0C6
:102A7D00C4F854F0C868FEA3E0C4540F48FFEE54E8
:102A8D000FFEC3648094885021EF25E0FFEE33FEE6
:102A9D0074A72FF58274063EF583E493FF740193BA
:102AAD00900302CFF0A3EFF0802BEE5407FEEF253D
:102ABD00E0FFEE33FE74A72FF58274063EF583E436
:102ACD0093FE740193FFC374FF9F900303F0740F83
:102ADD009E900302F0900237E0FEA3E0FF90030802
:0F2AED00E02FF0900307E03EF0758CFE758A1A1B
:0F2AFC00D007D006D000D0D0D082D083D0E03227
:031A1200022F9A06
:102F9A00C0E0C0F0C083C082C0D075D000C000C0FD
:102FAA0001C002C003C004C005C006C00753C87FE1
:102FBA00123146D007D006D005D004D003D002D0B3
:0E2FCA0001D000D0D0D082D083D0F0D0E03241
:103146009002F1E0F5BBE004F0E0D3648094904097
:103156000C7406F0122BCD1232E412331743E8102A
:013166002246
:07331700E51424FF92872258
:031A2100022DE8AB
:102DE800C0E0C0F0C083C082C0D075D000C000C0B1
:0D2DF80001C002C003C004C005C006C00732
:102E050053E8DFADBDAFBEEFFE7C00E42DFFEC3E29
:102E1500FEADBBED25E02406F582E43402F583EE34
:0E2E2500F0A3EFF09002F1E0B41003121A24B3
:102E3300D007D006D005D004D003D002D001D000F3
:0B2E4300D0D0D082D083D0F0D0E0329D
:101A240090021CE0FFA3E09002F6CFF0A3EFF09049
:101A3400021EE0FFA3E09002F8CFF0A3EFF09002C3
:101A440020E0FFA3E09002FACFF0A3EFF09002228F
:101A5400E0FFA3E09002FCCFF0A3EFF0900224E0BB
:101A6400FFA3E09002FECFF0A3EFF090023AE06013
:101A7400509002F6E0FFA3E0900394CFF0A3EFF0C0
:101A84009002F8E0FFA3E0900396CFF0A3EFF0906C
:101A940002FAE0FFA3E0900398CFF0A3EFF09002E6
:101AA400FCE0FFA3E090039ACFF0A3EFF09002FED6
:101AB400E0FFA3E090039CCFF0A3EFF0E490023AA0
:101AC400F07F0012214C7F0112214C7F0212214C25
:101AD4007F0312214C7F0412214CAF18AE17D3742C
:101AE400649F74089E5009EF249CFFEE34F7802213
:101AF400C3749C9F74079E5012C3EF9464EE9408C1
:101B04005009E4900326F0A3F0800EEF2464FFEE66
:101B140034F8900326F0A3EFF0900218E0FFA3E05E
:101B240090032ACFF0A3EFF0900216E0FEA3E0FFAB
:101B3400EE3395E0FDFCE42FFFEE34F8FEED34FFC8
:101B4400FDEC34FFFC90032C121FDE900326E0FE14
:101B5400A3E0FBAA06EA3395E0F9F890032AE0FE35
:101B6400A3E0FFEE3395E0FDFC121F4490031E1228
:101B74001FDEE4FB7A08F9F890031EE0FCA3E0FD05
:101B8400A3E0FEA3E0FF1219C2900322121FDEAEEF
:101B940015AF16E4FCFD90032CE0F8A3E0F9A3E0F4
:101BA400FAA3E0FB121F4490031E121FDEE4FB7A2B
:101BB40020F9F890031EE0FCA3E0FDA3E0FEA3E0FF
:101BC400FF1219C2900328EEF0A3EFF0AE19AF1A7A
:101BD4007C007D0A121F1CE4FD90031E121FDEE42C
:101BE4007B0BFAF9F890031EE0FCA3E0FDA3E0FEF2
:101BF400A3E0FF1219C2AB07AA06900322A3A3E035
:101C0400FEA3E02BFFEE3AFE9002EFF0A3EFF0D339
:101C140094FFEE6480948F400A9002EF740FF0A357
:101C240074FFF0C39002F0E094019002EFE064804E
:101C340094805005E4F0A304F09002EFE0FEA3E0EA
:101C4400FFEE3395E0FDFCE4FB7A0BF9F8121F4438
:101C540090031E121FDE90031EE0FCA3E0FDA3E030
:101C6400FEA3E0FFE4FB7A10F9F81219C290031EF8
:101C7400121FDE900322121FEA00000000E47F0B13
:101C8400FEFDFC900322E0F8A3E0F9A3E0FAA3E050
:101C9400FBC3121F934003021D34900322A3A3E04D
:101CA400FEA3E09018A775F00212201BEE25E02594
:101CB40083F583E493FE740193FF900326EEF0A36F
:101CC400EFF0EE3395E0FDFC90031EE0F8A3E0F99D
:101CD400A3E0FAA3E0FBC3121F93402C90031EA3BE
:101CE400A3E0FEA3E0FF900326E0FCA3E0FDEF9D4C
:101CF400FFEE9C900330F0A3EFF0900322A3A3A384
:101D0400E004900239F08028900322E0FCA3E0FD77
:101D1400A3E0FEA3E0FFE4FAF9F8EF2401FFEA3EB2
:101D2400FEE93DFDE83CFC900322121FDE021C810B
:101D3400900331E025E0FF900330E033FE74A72FD9
:101D4400F58274163EF583E493FE740193FF9002CA
:101D540039E0FDEFA805088005CEC313CE13D8F9EA
:101D6400FF900237EEF0A3EFF0900328E0FEA3E02B
:101D7400FF900238E02FF0900237E03EF0E4251C9B
:101D8400FFE51B34F8FE900326F0A3EFF0FBAA0650
:101D9400EA3395E0F9F8900226E0FEA3E0FFEE3383
:101DA40095E0FDFC121F4490031E121FDEE4FB7A33
:101DB40008F9F890031EE0FCA3E0FDA3E0FEA3E015
:101DC400FF1219C2E51E2FFFE51D3EFE9002F2F040
:101DD400A3EFF0D394FFEE6480948F400A9002F254
:101DE400740FF0A374FFF0C39002F2E06480948057
:061DF4005004E4F0A3F02E
:011DFA0022C6
:0D2EF6004A039400000000000000000000EE
:0E214C0090FFFF12204DEFF090FFEE12204D9D
:10215A00852283852382E4F0A3F090001212207175
:10216A00E025E02494F582E43403F583E0FEA3E05D
:10217A00FFFBAA06E4F9F8900012122071E075F04C
:10218A0002A424F6F582E5F03402F583E0FEA3E02A
:10219A00FFC3EF9BFFEE9AFEE499FDE498FC8522CB
:1021AA0083852382A3A3121FDEE47F08FEFDFC853C
:1021BA002283852382A3A3E0F8A3E0F9A3E0FAA38C
:1021CA00E0FBC3121F93400B852283852382E4F030
:1021DA00A304F074FF7FF8FEFDFC85228385238229
:1021EA00A3A3E0F8A3E0F9A3E0FAA3E0FBD3121F4C
:1021FA0093500B85228385238274FFF0A3F08522F6
:10220A0083852382E0FEA3E0FF4E7003022469EF78
:0A221A00F47002EEF46003022303E7
:10222400900012122071E025E02494F582E4340336
:10223400F583E0FEA3E0FFE4FCFD90000E122071A4
:10224400121FDEE47F01FEFDFC90000E122071E0FF
:10225400F8A3E0F9A3E0FAA3E0FBC3121F93500D27
:1022640090000E122071121FEA000000019000126B
:10227400122071E025E02415F8E6FE08E6FFE4FCF0
:10228400FD7BFF7A0FF9F8121F4490000E122071A3
:10229400E0F8A3E0F9A3E0FAA3E0FB1219C290006E
:1022A40006122071121FDE900012122071E075F0E8
:1022B40002A424F6F582E5F03402F583E0FEA3E0FF
:1022C400FFE4FCFD900006122071E0F8A3E0F9A3FE
:1022D400E0FAA3E0FB121F4490000A122071121FBF
:1022E400DEE47BFF7A0FF9F890000A122071E0FC1B
:0C22F400A3E0FDA3E0FEA3E0FF1219C26E
:10230000022429852283852382E0FEA3E064014E16
:05231000600302243D02
:10231500900012122071E025E02415F8E6FE08E68B
:10232500FBAA06C374FF9BFF740F9AFEE49400FD9D
:10233500E49400FCE47BFF7A0FF9F8121F44900047
:1023450006122071121FDE900012122071E025E0A6
:102355002494F582E43403F583E0FEA3E0FBC37423
:10236500FF9BFF740F9EFEE49400FDE49400FC9037
:10237500000A122071121FDEE47F01FEFDFC9000B1
:102385000A122071E0F8A3E0F9A3E0FAA3E0FBC389
:10239500121F93500D90000A122071121FEA0000BF
:1023A5000001900006122071C083C082E0FCA3E00A
:1023B500FDA3E0FEA3E0FF90000A122071E0F8A360
:1023C500E0F9A3E0FAA3E0FB1219C2D082D0831290
:1023D5001FDE900012122071E075F002A424F6F5BC
:1023E50082E5F03402F583E0FEA3E0FBC374FF9BB6
:1023F500FF740F9EFEE49400FDE49400FC9000063B
:10240500122071E0F8A3E0F9A3E0FAA3E0FB121FA4
:1024150044E47BFF7A0FF9F81219C2C374FF9FFFDA
:10242500740F9EFE900012122071E025E02415F82D
:08243500A60608A6071232D525
:10243D00900012122071E0FF75F002A424F6F582CF
:10244D00E5F03402F583E0FCA3E0FDEF25E02494F4
:0C245D00F582E43403F583ECF0A3EDF00D
:0624690090001302204D5B
:011A1100FFD5
:022F0300C10CFF
:102E4E00E490030AF0FB7A00791490030F121FEA44
:102E5E000000000BE4FD1230DD75170875180075C3
:102E6E001B08751C00123308E4900309F090030947
:102E7E00E0FFC3941E502A75F00BEFA42400F582D8
:102E8E00E5F0343AAF82FE7B007A0079149003109D
:102E9E00E4F0A3740BF0122F54900309E004F080B9
:042EAE00CC02309290
:0F32D500200C099002F4E06003121A09D20C22B7
:10325900901A11E493600C122E4E7E1A7F11E4FD30
:09326900123167E49003B0F02279
:103124009003B0E075F00BA42400F9743A35F0FA7A
:103134007BFF78147C007D007E007F0B121ECBC2C7
:023144000C225B
:10303D001233089003B0E075F00BA42400F582E57F
:10304D00F0343AAF82FE7B007A007914900310E4DD
:0B305D00F0A3740BF0122F540230920D
:061A1B0012303DC20C2256
:0A264400900371EDF0900370EFF0C9
:10264E00D39B5003022722E024FFFEE434FF9003C5
:10265E0075F0A3CEF0EB14900374F0900371E024A8
:10266E00FFFFE434FFFE900375E0FCA3E0FDD39F73
:10267E00EE6480F8EC64809840030227F3903A00F1
:10268E0075F00BED12201BEC75F00BA42583AF82B9
:10269E0090037CF0A3EFF0900374E075F00BA4248C
:1026AE0000F9743A35F0FA90037974FFF0A3EAF06A
:1026BE00A3E9F0E4900377F0A3F0900379A3E47517
:1026CE00F001121F2EFEAFF090037CE475F00112A4
:1026DE001F2E85F082F583E493FD122C5F90037814
:1026EE00E004F07006900377E004F0C3900378E006
:1026FE00940B900377E0940040C0123092900376D2
:10270E00E004F07006900375E004F0900374E004AA
:10271E00F0022669900371E024FFFEE434FF90037B
:10272E0075F0A3CEF0900373E014A3F0900370E065
:10273E0024FFFFE434FFFE900375E0FCA3E0FDC32D
:10274E009FEE6480F8EC64809850030227F3903A71
:10275E000075F00BED12201BEC75F00BA42583AF6A
:10276E008290037CF0A3EFF0900374E075F00BA45D
:10277E002400F9743A35F0FA90037974FFF0A3EA65
:10278E00F0A3E9F0E4900377F0A3F0900379A3E4CB
:10279E0075F001121F2EFEAFF090037CE475F00170
:1027AE00121F2E85F082F583E493FD122C5F9003A9
:1027BE0078E004F07006900377E004F0C39003789D
:1027CE00E0940B900377E0940040C0123092900397
:1027DE0076E024FFF0900375E034FFF0900374E090
:0527EE0014F002273A7F
:0127F30022C3
:0527F40090035BEDF015
:1027F900EF1490036CF0EB14A3F090035BE014FF6B
:1028090090036CE0D39F4003022953A3E075F00BBA
:10281900A42400F582E5F0343AAF82FEE490036E19
:10282900F0A3F090036EE0FCA3E0FDC3940BEC94DD
:1028390000502B0FEFAA0670010E14F5828A83E46B
:1028490093FB74612DF582E43403F583EBF0900377
:102859006FE004F070CD90036EE004F080C5900342
:102869006DE075F00BA42400F9743A35F0FA900381
:102879005C74FFF0A3EAF0A3E9F090036CE075F053
:102889000BA42400F582E5F0343AAF8290035FF09F
:10289900A3EFF0E490036EF0A3F090035CA3E4755A
:1028A900F001121F2EFEAFF090035FE475F00112E4
:1028B9001F2E85F082F583E493FD122C5F90036F40
:1028C900E004F0700690036EE004F0C390036FE03B
:1028D900940B90036EE0940040C090036CE075F097
:1028E9000BA42400F9743A35F0FA90035C74FFF0F4
:1028F900A3EAF0A3E9F0E490036EF0A3F090036E6D
:10290900E0FCA3E0FDC3940BEC9400502D90035C14
:10291900A3E475F001121F2EFEAFF074612DF5824C
:10292900E43403F583E0FD122C5F90036FE004F0BB
:1029390070CB90036EE004F080C312309290036C68
:0A294900E004F0A3E004F00228030C
:012953002261
:072B0B0090037EEBF0AC0724
:102B1200A3E5C1F0A2AFE433A3F0AF05A3E4F0A3B1
:102B2200EFF0E07F00FE900381F0A3EFF0AD04ED43
:102B3200FF900381EEF0A3EFF0C2AF900387740F12
:102B4200F0123308900387E075F00BA42400F974A7
:102B52003A35F0FA90038374FFF0A3EAF0A3E9F0A8
:102B6200E4A3F0900381E0FCA3E0FFECFD90037E80
:102B7200E0FBE49003A8F0D2001218BD900388EFA6
:102B8200F0FD900383A3E475F001121F2EFEAFF057
:102B9200122C5F900382E004F07006900381E0043F
:102BA200F0900386E004F0E0C3940B40B61230923A
:102BB200900387E004F0E0C3941E408590037FE019
:0B2BC200F5C1A3E024FF92AF02331E18
:07295400900389EBF0AC07D2
:10295B00A3E5C1F0A2AFE433A3F0AF05900390E47D
:10296B00F0A3EFF0E07F00FE900390F0A3EFF0AD4B
:10297B0004EDFF900390EEF0A3EFF0C2AF90038E47
:10298B00E4F0A3740FF090038EE0FEA3E0FFC3947A
:10299B001EEE94004003022A2D903A0075F00BEFC7
:1029AB0012201BEE75F00BA42583AF82900392F0DF
:1029BB00A3EFF0E490038CF0A3F0900390E0FCA362
:1029CB00E0FFECFD900389E0FB900392E475F001CE
:1029DB00121F2E85F082F583E4939003A8F0C200BA
:1029EB001218BD900391E004F07006900390E00480
:1029FB00F090038DE004F0700690038CE004F0C3BC
:102A0B0090038DE0940B90038CE0940040AC90030A
:102A1B008FE004F0600302299190038EE004F00232
:102A2B00299190038AE0F5C1A3E024FF92AF023312
:012A3B001E7C
:03000000020600F5
:03000300021A03DB
:03000B00021A06D0
:03001300021A09C5
:03001B00021A0CBA
:03002300021A0FAF
:03002B00021A12A4
:03003300021A1599
:03003B00021A188E
:03004300021A1B83
:03004B00021A1E78
:03005300021A216D
:03005B00021A2462
:03006300021A2757
:03006B00021A2A4C
:03007300021A2D41
:10060000E4F5D9E5EF7480F5FF7402F5EF787FE447
:10061000F6D8FD9000007F007E08E4F0A3DFFCDE4A
:07062000FA75812302066256
:1031880090031CEFF0A3EDF07F0A122CED90031CC6
:10319800E0FF122CED90031DE0FF122CED02331E10
:081A09007F02122CED02331ED6
:06300D00123325EF6027DD
:103013009003097403F0A3749EF0123068900309BF
:10302300E475F001121F2E85F082F583EFF0123361
:073033002BEF70E67F012284
:03303A007F0022F2
:10328A009003B1EFF07F2F122CED9003B1E0FF1203
:05329A002CED02331EC3
:10329F009003B2EFF07F30122CED9003B2E0FF12EB
:0532AF002CED02331EAE
:022F0500C10900
:10327200E50BB50FFBE50AB50EF6E50BB513F1E567
:083282000AB512EC20C5E92297
:0C32F200438E08758D5D858D8BD28E2279
:1032B40075C101E4F5C2F5C053C17F43C180023238
:0132C400F217
:1030B8007E037F338E0C8F0D8E108F118E088F0933
:1030C8007E037F478E0E8F0F8E128F138E0A8F0B03
:0530D800C2080232B441
:102FD8000511E511AA107002051014F5828A83EF15
:102FE800F0AF050511E511AC107002051014F5825B
:102FF8008C83EFF07447B5110B7403B51006751088
:053008000375113322E5
:07331E00C208C2C4D2C5229F
:102CED00200845D2080513E513AC12700205121425
:102CFD00F5828C8374FFF07C037D5BEDB5130AECDC
:102D0D00B512067512037513470513E513AA127054
:102D1D0002051214F5828A83E4F0EDB5130AECB5C1
:102D2D0012067512037513470513E513AC127002E5
:102D3D00051214F5828C83E4F07C037D5BEDB513F5
:102D4D000AECB512067512037513470513E513AAA0
:102D5D00127002051214F5828A83EFF0EDB5130A95
:0D2D6D00ECB512067512037513477F0122A5
:10320500E509B50D08E508B50C037F0022850D829B
:0D321500850C83E0B507037F01227F0022B6
:10306800050DE50D7002050C050DE50DAE0C7002A1
:10307800050C14F5828E83E0FF7447B50D0B7403BD
:09308800B50C06750C03750D333F
:01309100221C
:063325007FFF12320522B9
:06332B00E4FF123205224E
:031A180002246F36
:10246F00C0E0C083C082C0D075D000C000C002C021
:07247F0004C005C006C00700
:10248600E5C054FE122027260B08260B0A26210C2F
:1024960026210E25EA1025EA1225FD1425FD16250E
:1024A600E21C25E21E25DE2425DE26259F28259F03
:1024B6002A25AD2C25AD2E259642259644259646F1
:1024C6002596502596522596542596562596882566
:1024D600968A2524C02531C224E8E024E8E20000DB
:1024E600262DC2C5050BE50B7002050A7E037F5B30
:1024F600B5070AEEB50A06750A03750B47050BE51F
:102506000BAC0A7002050A14F5828C83E0F5C2EF63
:10251600650B7003EE650A600302262D8069850E41
:102526000A850F0BD2C4D2C502262DE50BB51312B0
:10253600E50AB5120D85120E85130FC2C5D2C40267
:10254600262D850B82850A83E0B4FF030226290522
:102556000BE50B7002050A7E037F5BB5070AEEB535
:102566000A06750A03750B47050BE50BAC0A7002E4
:10257600050A14F5828C83E0F5C2EF650B7003EE55
:10258600650A600302262D750A03750B4702262D80
:10259600900332E004F002262DE5C2602A9002F58F
:1025A600E065C260228016850E0A850F0BC2C5D271
:1025B60009E5C260129002F5E065C2600AC2C4C2B3
:1025C600C5C2C1C20A8060ADC27FFF122FD8C2C485
:1025D600C2C5D2C1D20A804FD2C5804B850A0E85AC
:1025E6000B0F8043851008851109C2C4C2C130098A
:1025F60036D2C5C2098030850E0A850F0BC2C4C209
:10260600C1D2C58022C2C4C2C5200A04C2C1801775
:10261600ADC2E4FF122FD8D2C1800C850E0A850FF9
:092626000BC2C1C2C4D2C5C2C07E
:10262F00D007D006D005D004D002D000D0D0D082B1
:05263F00D083D0E03261
:0530DD0090030EEDF070
:1030E20090030F74FF121FABEC4D4E4F6010900314
:0E30F2000EE0121F0A740129F9E43AFA80E296
:0131000022AC
:1031A800A2AFE433FDC2AF758F0375B7A575B7F14C
:0F31B8008F828E83E4F0F58FAF05EF24FF92AF87
:0131C70022E5
:10316700A2AFE433FCC2AF758F0175B7A575B7F190
:103177008F828E83EDF0E4F58FAF04EF24FF92AFDB
:013187002225
:102F0800900318EEF0A3EFF0A3ECF0A3EDF0EB4A7A
:102F18006039900318E0FEA3E0FFA3E0FCA3E0F50E
:102F2800828C83E0FD123167EB1B70011A90031B42
:102F3800E004F0700690031AE004F0900319E0042E
:0C2F4800F070CB900318E004F080C3226E
:08330800E4900000F0A3F022A4
:10309200900000E0FEA3E0FF1231A8900000E0FEE5
:1030A200A3E0FF7C007D027B007A02122F08E490ED
:0630B2000000F0A3F02273
:0A2C5F00A905900312EEF0A3EFF0B8
:102C6900EE54FEFE900000E0FCA3E0FD7002EE6C65
:102C79006059ED4C6003123092900312E0FEEE545D
:102C8900FEFE7F00900000F0A3EFF0900314EEF039
:102C9900A3EFF0A37400F0A37402F07F007E02900A
:102CA9000314E475F001121F2E85F082F583E49375
:102CB900FD900316E475F001121F2E85F082F5834D
:102CC900EDF0EF1F70011EEF4E70D4900312E0FC7F
:102CD900A3E0FDEC5401FC74022DF58274003CF56F
:032CE90083E9F08C
:012CEC0022C5
:102F540090030BEEF0A3EFF0A3EBF0A3EAF0A3E9E8
:102F6400F090031074FFF5F0121F2E45F0602690C8
:102F7400030BE475F001121F2EAFF0FE90030DE079
:102F8400FBA3E475F001121F2EA9F0FA121EF1FD45
:062F9400122C5F80CC222C
:0818BD009003A5EFF0A3EDF08C
:1018C500A2009204C206200DFDD20D9003A9EBF0F3
:1018D500C201D202D2057F01C2C4C207D2C530C03F
:1018E500FDE5C054F02480700302197724C0601B05
:1018F50024E060030219A79003A9E0F5C2A201E460
:101905003342C2C2C5E4A3F00219A930C159300758
:1019150007D2C5C2070219A930020CC202D2039030
:1019250003A6E0F5C2807D300311C2039003A5E054
:10193500F5C230046FD207D2018069200166EFFD40
:101945009003AAE0FB3395E0FAC3EB9D7480F86A37
:1019550098500E9003A8E0F5C29003AAE004F08029
:1019650043D2C4C20D803D300504D2C58036D206AF
:101975008032EFFD9003AAE0FB3395E0FAC3EB9DBF
:101985007480F86A98500CA3E5C2F09003AAE004AD
:10199500F0D2C19003AAE0B5070AC20DC2C1D2C4F4
:1019A5008002D20630060853C0BF43C040C20DC2F4
:0C19B500C0300D030218E39003ABE0FF0C
:0119C1002203
:10062700022D7AE493A3F8E493A34003F68001F242
:1006370008DFF48029E493A3F85407240CC8C333D4
:10064700C4540F4420C8834004F456800146F6DFA3
:10065700E4800B0102040810204080902EB2E47E53
:10066700019360BCA3FF543F30E509541FFEE49398
:10067700A360010ECF54C025E060A840B8E493A35F
:10068700FAE493A3F8E493A3C8C582C8CAC583CA8A
:10069700F0A3C8C582C8CAC583CADFE9DEE780BE42
:012F070000C9
:101DFB00E709F608DFFA8046E709F208DFFA803ECA
:101E0B0088828C83E709F0A3DFFA8032E309F608B6
:101E1B00DFFA8078E309F208DFFA807088828C831E
:101E2B00E309F0A3DFFA806489828A83E0A3F608D2
:101E3B00DFFA805889828A83E0A3F208DFFA804CAC
:101E4B0080D280FA80C680D4806980F28033801083
:101E5B0080A680EA809A80A880DA80E280CA8033EC
:101E6B0089828A83ECFAE493A3C8C582C8CCC58364
:101E7B00CCF0A3C8C582C8CCC583CCDFE9DEE78034
:101E8B000D89828A83E493A3F608DFF9ECFAA9F0B3
:101E9B00EDFB2289828A83ECFAE0A3C8C582C8CC09
:101EAB00C583CCF0A3C8C582C8CCC583CCDFEADE22
:101EBB00E880DB89828A83E493A3F208DFF980CC84
:101ECB0088F0EF60010E4E60C388F0ED2402B4047D
:101EDB000050B9F582EB2402B4040050AF23234524
:061EEB008223901E4B73E0
:101EF100BB010689828A83E0225002E722BBFE02EF
:091F0100E32289828A83E4932221
:101F0A00BB010689828A83F0225002F722BBFE01B6
:021F1A00F322B0
:101F1C00EF8DF0A4A8F0CF8CF0A428CE8DF0A42ED9
:021F2C00FE2293
:101F2E00A3F8E0C5F025F0F0E58215827002158366
:061F3E00E0C838F0E822C3
:101F4400E88FF0A4CC8BF0A42CFCE98EF0A42CFC3C
:101F54008AF0EDA42CFCEA8EF0A4CDA8F08BF0A4BA
:101F64002DCC3825F0FDE98FF0A42CCD35F0FCEB19
:101F74008EF0A4FEA9F0EB8FF0A4CFC5F02ECD39DE
:0F1F8400FEE43CFCEAA42DCE35F0FDE43CFC224B
:1019C200C2D5E830E70FB2D5E4C39BFBE49AFAE450
:1019D20099F9E498F8EC30E717B2D51219F8122009
:1019E200BAE4C39BFBE49AFAE499F9E498F8800319
:1019F2001220BA30D50DE4C39FFFE49EFEE49DFDA4
:041A0200E49CFC2242
:101F9300EB9FF5F0EA9E42F0E99D42F0EC6480C8C5
:061FA30064809845F02265
:101FA9007401FF3395E0FEFDFCA3A3A3E0CF2FF05E
:101FB900E582158270021583E0CE3EF0E582158236
:101FC90070021583E0CD3DF0E5821582700215831C
:051FD900E0CC3CF02209
:0C1FDE00ECF0A3EDF0A3EEF0A3EFF02276
:101FEA00A8828583F0D083D08212200112200112A8
:101FFA002001122001E473E493A3C583C5F0C583CD
:10200A00C8C582C8F0A3C583C5F0C583C8C582C840
:01201A0022A3
:0C201B00A42582F582E5F03583F58322D0
:10202700D083D082F8E4937012740193700DA3A348
:1020370093F8740193F5828883E47374029368605C
:06204700EFA3A3A380DF5C
:10204D00E5232582F582E5223583F583B5220485C6
:10205D0082232210AF06858223F52222858223F565
:04206D0022D2AF22AA
:0D207100E5232582F582E5223583F58322E3
:10207E0075F008758200EF2FFFEE33FECD33CDCC19
:10208E0033CCC58233C5829BED9AEC99E58298409C
:10209E000CF582EE9BFEED9AFDEC99FC0FD5F0D679
:1020AE00E4CEFBE4CDFAE4CCF9A88222B800C1B9A3
:1020BE000059BA002DEC8BF084CFCECDFCE5F0CBE1
:1020CE00F97818EF2FFFEE33FEED33FDEC33FCEB1A
:1020DE0033FB10D703994004EB99FB0FD8E5E4F9D5
:1020EE00FA227818EF2FFFEE33FEED33FDEC33FCC2
:1020FE00C933C910D7059BE99A4007EC9BFCE99AB6
:10210E00F90FD8E0E4C9FAE4CCFB2275F010EF2FFA
:10211E00FFEE33FEED33FDCC33CCC833C810D707FA
:10212E009BEC9AE899400AED9BFDEC9AFCE899F835
:0E213E000FD5F0DAE4CDFBE4CCFAE4C8F922C8
:00000001FF
